:020000040800F2
:10000000E81B0020010100080B0E0008510C00083D
:10001000090E000861090008D5150008000000005D
:10002000000000000000000000000000D50E0008E5
:100030006309000800000000D30E000869140008DE
:100040001B0100081B0100081B0100081B01000820
:100050001B0100081B0100081B0100081B01000810
:100060001B0100081B0100081B0100081B01000800
:100070001B0100081B0100081B0100081B010008F0
:100080001B0100081B0100081B0100081B010008E0
:100090001B0100081B0100081B0100081B010008D0
:1000A0001B0100081B0100081B0100081B010008C0
:1000B0001B0100081B010008000000001B010008D4
:1000C0001B01000800000000000000001B010008E8
:1000D00000000000311500081B01000800000000AE
:1000E0001B0100081B0100081B010008DFF80CD0F1
:1000F00000F040F90048004751160008E81B0020B6
:100100000648804706480047FEE7FEE7FEE7FEE7B1
:10011000FEE7FEE7FEE7FEE7FEE7FEE7E514000880
:10012000ED00000830B50B460146002020220124D6
:1001300009E021FA02F59D4205D303FA02F5491BB5
:1001400004FA02F52844151EA2F10102F1DC30BDCB
:100150002DE9F05F0546002092469B4688460646FC
:10016000814640241BE0284641464746224600F08F
:1001700022F953465A46C01A914110D311461846E7
:10018000224600F009F92D1A67EB01084F46224676
:100190000120002100F000F917EB00094E41201E5C
:1001A000A4F10104DFDC484631462A464346BDE857
:1001B000F09F2DE9FE4F81EA030404F0004421F092
:1001C000004100944FF0000B23F0004350EA01047B
:1001D0005ED052EA03045BD0C3F30A54C1F30A555C
:1001E0002C44A4F2F3340194A0FB0254C1F3130194
:1001F00041F48011C3F3130343F4801301FB024461
:1002000000FB034E840A970A44EA815447EA835765
:10021000A4FB076802958D0A05FB07854FEA932C1E
:1002200004FB0C542705029D4FEA065847EA16378F
:10023000B5EB08056EEB070C870E920E47EA8117A7
:1002400042EA8312A7FB0201B6EB0B0164EB000448
:100250002B0D43EA0C335E1844EB1C50DA46514632
:10026000E7FB0201C5F313044FEA0B3343EA1453CF
:100270004FEA0432019C43EA0603A4F10C04029401
:10028000009CCDE900B400F0B5F803B0BDE8F08FF4
:1002900000200146F9E72DE9F04D81EA030404F05E
:1002A000004B21F0004514464FF0000A23F00041B6
:1002B00050EA050220D054EA01021DD0C5F30A57C6
:1002C0000246C5F31303C1F31300C1F30A5640F409
:1002D000801543F48013A7EB0608101BD64608F2DE
:1002E000FD3873EB050002D308F1010801E0921814
:1002F0005B41B8F1000F03DA00200146BDE8F08D44
:1003000000204FF48011064684460EE0171B73EB65
:10031000050705D3121B63EB050306434CEA010CEA
:1003200049084FEA300092185B4150EA0107EDD1CD
:1003300052EA030012D082EA040083EA050108436E
:1003400005D0101BAB4106D20122002306E000229B
:100350004FF0004302E06FF0010253101AEB060069
:100360004CEB085110EB0A0041EB0B01BDE8F04DDE
:1003700000F031B8064C074D06E0E06840F001039C
:1003800094E8070098471034AC42F6D3FFF7B2FE6A
:100390002020000840200008202A04DB203A00FA30
:1003A00002F1002070479140C2F1200320FA03F3CC
:1003B000194390407047202A04DB203A21FA02F0CA
:1003C0000021704721FA02F3D040C2F1200291408F
:1003D00008431946704710B5141E73F1000408DA7B
:1003E000401C41F1000192185B411A4301D120F0F9
:1003F000010010BD2DE9F04D92469B4611B1B1FAB6
:1004000081F202E0B0FA80F220329046FFF7C4FF9A
:1004100004460F4640EA0A0041EA0B0153465A4699
:10042000084313D0114653EA010019D0C8F1400225
:100430005046FFF7C0FF05460E4650465946424615
:10044000FFF7AAFF084305D0012004E02046394603
:10045000BDE8F08D0020054346EAE0762C433743A3
:100460000A986305E40AA0EB08000022FD0A44EAAA
:1004700047540A3002D500200146E9E7010510196A
:100480006941DDE9084500196941BDE8F04DA2E781
:1004900040EA01039B0703D009E008C9121F08C006
:1004A000042AFAD203E011F8013B00F8013B521E86
:1004B000F9D27047D2B201E000F8012B491EFBD2FD
:1004C00070470022F6E710B513460A46044619465F
:1004D000FFF7F0FF204610BDF0B480EA0102D40F10
:1004E0004200B2EB410F02D20246084611464A00D2
:1004F00042D0C30DDDB2C1F3C752AD1A202D35DA9B
:10050000C1F3160141F4000204B15242C5F12006C4
:1005100002FA06F12A411044B3EBD05F23D0C4B1F4
:10052000012DA0EBC35009DCF0BC4FF0004202EA01
:10053000C352DBB200F5000000F0DCB8400000F16F
:10054000807000EBC350A0F1807040EAD170490088
:1005500009E0490841EAC071A0EBC35000F5000072
:10056000400800EBC350F0BC00F0BBB86142012270
:1005700002EB4101001BF6E7F0BC704781F000413F
:10058000AAE780F00040A7E780EA010210B502F078
:100590000043400022D04A001FD0010E01EB12613F
:1005A000C0F35600C2F3560240F4000042F40002C9
:1005B000A0FB022000047F39140400D0401C50EA44
:1005C000124001D44000491EC2B20C0604EBD01008
:1005D000401C4008802A02D003E0002010BD20F01B
:1005E0000100002900DA0020184310BD30B480EA71
:1005F000010202F0004530F0004221F0004013D02B
:1006000090B1C30DD40DC2F31601C0F31600E41A65
:1006100041F4000140F400027D34914201D3641C96
:1006200000E04900002C02DA30BC002070474FF493
:1006300000000023914201D3891A034340084FEA86
:100640004101F7D151B1914202D14FF0004105E093
:1006500002D24FF0010101E06FF0010103EBC45041
:10066000284430BC00F03DB8C10F80EAE070084477
:10067000CA079623002100F03DB8962300221146B8
:1006800000F038B800F0004230F000400AD0C10D50
:1006900001F56071C0F3160042EA0151C20840073B
:1006A0001143704700200146704701F0004330B409
:1006B00021F0004150EA010206D00A0DA2F5607255
:1006C000C1F31301002A02DC30BC00207047440F44
:1006D00044EAC104C100E01830BC00EBC250AFF3E3
:1006E00000800029A8BF7047401C490008BF20F0C7
:1006F0000100704710B4B0FA80FC00FA0CF050EA28
:10070000010404BF10BC704749B1CCF1200421FAA8
:1007100004F411FA0CF118BF012121430843A3EBA3
:100720000C01CB1D4FEA00614FEA102042BF0020B0
:1007300010BC704700EBC35010440029A4BF10BC8C
:100740007047401C490008BF20F0010010BC7047F2
:100750002DE9FE4F0D460646002400F085F840B214
:10076000B0F1FF3F08DC012000F0FCF8601C632CB6
:100770000446F2D9BDE8FE8F824800F096FB204681
:10078000712100F0B5FD00F09BFB304F2046B847CB
:1007900001962F4E2046B0472046B8478046204657
:1007A000B0472046B847029505462046B047204648
:1007B000B84781462046B0472046B8478246204683
:1007C000B0472046B8478346204600F0F5FC204657
:1007D00000F056FD280240EA084048440009FFF7AF
:1007E0004CFFFFF74FFF1B4B0022FFF7E2FC1A4CB8
:1007F00000222346FFF7DDFC00222346FFF7D9FC49
:10080000FFF753FF019908604FF4702000EA094098
:1008100040EA0A205844FFF730FF1049FFF7B4FEC2
:100820000F4C2146FFF7B0FE4FF06A51FFF7ACFEC8
:100830004FF06A51FFF7A8FE0A49FFF74DFE214627
:10084000FFF7D4FE02990860BDE8FE8FD9110008B9
:10085000E9100008000059400000503F00004843E4
:10086000000020410000FAC3B0B5E44800F01DFBD1
:100870002046712100F03CFD00F022FB204600F0F4
:10088000ABFC0546204600F097FC204600F0F8FC43
:100890002846B0BD70B5D94800F007FB0D4D204685
:1008A0007021A8470C4E2046B0472046AC21A847EF
:1008B0002046B04720463321A8472046B04720466F
:1008C0000021A8472046B0472046BDE8704000F010
:1008D000D7BC00BFF1120008A512000870B5C748C8
:1008E00000F0A7FA2046472100F002FD00F0E8FAE8
:1008F000204600F071FC0546204600F0F5FB20463E
:1009000000F06AFC0646204600F056FC204600F047
:10091000B7FC46EA0520FFF7A7FEFFF7B3FE044B3E
:100920004FF03332FFF7B7FCFFF7BFFE70BD00BFDB
:100930003333F33F10B5B14800F07BFA204646212F
:1009400000F0D6FC00F0BCFA2046102100F0D0FCEC
:1009500000F0B6FA2046BDE8104000F091BC00BFA0
:10096000FEE77047012181F31088A449012808BFE0
:10097000022048610020887080F310888878012860
:10098000FCD1704720050020B0B50B49984B0B4CAB
:100990000A681B68B3FBF4F34C68584300234D68A6
:1009A000AC42FCD023445B1BAC4298BF13442C46A2
:1009B000834228BFB0BDF2E714E000E040420F00E0
:1009C000024602A00BA101F0F5F9FEE74572726F35
:1009D00072206F636375727265643A2066696C6534
:1009E000202573206F6E206C696E652025640D0ACA
:1009F000000000002E2E2F53797374656D2F7379CC
:100A0000732F7379732E63002DE9FC4F5C4A032327
:100A10004FF0000A4FF001084FF00F0C4FF00009A3
:100A2000904208BF0223009300250B6833FA05F2B9
:100A300008BFBDE8FC8F08FA05FE13EA0E0F00F0B0
:100A40009A804F68032F16D9112F26D0122F28D045
:100A50004F4A974213D04F4A974210D04E4A97427E
:100A60000DD04E4A97420AD04D4A974207D04D4A80
:100A7000974204D022E0DFE807F002181B1F8B68C2
:100A800043B1012B14BFC0F814E0C0F810E04FF0E0
:100A9000080913E04FF0040910E0CB6803F10409E2
:100AA0000CE0CB6803F10C0908E0D1F80C9005E0EC
:100AB000CB6803F1080901E04FF0000953460646F0
:100AC000082D28BF203B28BF043637680CFA03F4F2
:100AD00009FA03F327EA040423433360CB79DB06E6
:100AE00049D52A4AAF08136843F00103136013681D
:100AF000244A03F00103A2F57E742B4A0193019B63
:100B000054F827B0904205D0284A009B904208BF75
:100B1000012300E000230AF00C060F2202FA06FC73
:100B2000B3402BEA0C024FF00F0C1A4344F8272075
:100B3000144C4F68FA03226854BF22EA0E0342EABB
:100B40000E032360BA03626854BF22EA0E0342EA2E
:100B50000E036360FA02A26854BF22EA0E0342EA5F
:100B60000E03A360084BBA021A6854BF22EA0E02B1
:100B700042EA0E021A600AF1040A013555E700BF85
:100B800000100140000401400C0401401810024014
:100B900000001110000012100000211000002210AF
:100BA000000031100000321000080140000C01402C
:100BB00010B50F494FF47A720968B1FBF2F14A1E81
:100BC0000021B1EB126F12D10A4BF0245A600A4A8D
:100BD0001470996007210F28196008D84FF0FF3072
:100BE0000F21002200F00CF8D4480121017010BD43
:100BF0000400002010E000E023ED00E020050020CC
:100C0000F0B5114B4FF0FF361C68C4F30224E51E0B
:100C100084F0070438BF002506FA05F7BA43042C10
:100C200028BF042406FA04F4A14300F00F04A940ED
:100C3000043C11432344054A09010C33B0F1FF3F42
:100C4000C8BF83181970F0BD0CED00E000E400E0AF
:100C5000FEE700002DE9F047DFF88498804699F818
:100C60000400E8BB664CFF20607500F06DF9F84D9C
:100C70004D208421A8472420FF21A847402001219E
:100C8000A84711203F21A84700F05AF92220FF2150
:100C9000A8470F2000F036F901460D20A847012093
:100CA0008D21A847324D002084F81701182000F04C
:100CB00029F9400705D455B10120FFF753FE01354E
:100CC000F4E7012089F804000320A07508E02068FB
:100CD00000F0D2F900F038F999F80400012842D167
:100CE000DFF800A49AF8110020B1132000F00AF9EF
:100CF000074601E09AF81570AFB30AF117044FF4F4
:100D000080712046FFF7DDFB102000F0FBF8014664
:100D10000D2000F003F9D9F80C00D0E9061000040A
:100D20000861002000F0BEF93E4625462EB100F0D5
:100D3000C3F905F8010B013EF8E7D9F80C008AF871
:100D400017718169808B086100F0FAF89AF81771C1
:100D500000264FB1404621463A46FFF799FB8AF8F4
:100D600017613E4600E000263046BDE8F08700BF30
:100D700019FCFFFF70B5DB4D044614200021687597
:100D8000D248017100F0E0F8B14E4D208721B04704
:100D900024200021B04740204121B04700F0D0F886
:100DA0001120F721B04722201421B0470E2000F077
:100DB000A9F801460D20B047124E222000F0A2F8FB
:100DC000142808D00136F8D3286800F055F9BDE89A
:100DD000704000F0B9B8022021461422A875002006
:100DE00000F07AF801208B2100F098F8122000F032
:100DF00089F800F0A5F8BDE8704000F069B900BFBF
:100E00000804002018FCFFFFFEE770470190032054
:100E1000CDE90212059000200490019870472069E6
:100E2000A168A2890A61FFF7AFBD0122002300F08B
:100E300083BA00F12C04204600F008BA22690904A4
:100E40000161500028474FF40052086880044FF0B9
:100E500008007047D4E902010904016110BD019046
:100E60000320059002A80EC001987047E08ED4E9D7
:100E70000912105C4860E08E0130E08680B2218E5D
:100E8000884270470A5003212322322340200090D9
:100E9000504600F08FBF40F004007061706900F0B0
:100EA0000400039003987069704700F1180420460D
:100EB00000F0CCB9A0682169A289026148002847E6
:100EC000204600F0EFB9D1E906210904116100F0D4
:100ED000E9B870477047000070B57C4E0D46144667
:100EE00040F08000F168FFF7EEFF2CB115F8010B20
:100EF00000F0D8F8013CF8E7F0688169808B086160
:100F000070BD00BF80B500F0CDF800F0D5F86F4996
:100F1000C9688A69898B116180BD00BFB0B56B4D0E
:100F20000C4640F08000E968FFF7CDFF204600F056
:100F3000B9F8E8688169808B0861B0BD20050020A0
:100F40001220FF21FFF7EABF7CB5414C01200821A8
:100F5000A047404D0020A8750F20FFF703FD01209A
:100F60008821A047D5E902013B4A0023C90441EA90
:100F70005031C004FFF7ECF8010A8DF80700000CAF
:100F800003228DF806108DF805000DF105010620ED
:100F9000FFF7A2FF39203421A047287C2FA1095C4C
:100FA0000920A0470B200B21A0470C202321A0479C
:100FB000A87C2BA3EA7C697C185C2CA39A5C520069
:100FC00002EB001089B1C1B21D20FFF7A7FF687CBA
:100FD000274A297D105C274A515C890001EB0010EB
:100FE000C1B21E20FFF79AFF1CE040F00100C1B221
:100FF0001D20A047687C1E4A297D105C1D4A515C5B
:10100000890001EB00100330C1B21E20A04731203F
:10101000FFF778FF00F0F800411D3120A04737208E
:101020000C21A04726200421A0471F200821A0470B
:10103000202000210026A04721200821A047412090
:101040000121A04785F81761BDE87C4000F040B859
:101050001D0F0008080400200048E801FFFCF9F615
:101060000001020304050607080900000102030449
:10107000D01F0008D71F000810B504461348C068E9
:101080008169808B0861D4E90001000408610120B6
:10109000FFF768FC6068218801616420BDE81040AA
:1010A000FFF760BC0146EF48C068D0E906231B0487
:1010B000136100F091B900BFEA48C068D0E9061298
:1010C00012040A61002100F087B900BF200500204A
:1010D00010B5012009210124FFF720FF0148847584
:1010E00010BD00BF0804002010B504460068231D91
:1010F0000ECB1B040904136101612069FFF744FC56
:10110000FFF78DFEFFF7A6BEFEB5B04B18444FEAC1
:10111000B02003280FD8DFE800F002101E2CAC48E6
:10112000036843F004030360006800F00400FFF765
:101130006DFEA8482AE000202CE0A548036843F093
:1011400008030360006800F00800FFF75FFEA14895
:1011500000F580601AE09E48036843F010030360C6
:10116000006800F01000FFF751FE9A4800F500609B
:101170000CE09748036843F020030360006800F028
:101180002000FFF743FE934800F5406002A9FFF7F7
:101190003BFC012006B080BD10B50446006811225A
:1011A0006168FFF7B1FF30B1D4E902010122BDE867
:1011B0001040FFF7A9BF10BD10B5D0E902230446C7
:1011C000016800691B041361A2880A61FFF7DCFB58
:1011D000FFF725FEFFF73EBE70B504460068616864
:1011E00000F01FF800260025072E14D8D4E90212BB
:1011F000206912040A61FFF7C7FBFFF710FED4E96C
:1012000000018068084080B2002818BF012040EA31
:1012100045050136E8E7D4E9000100F00CF8E8B232
:1012200070BDF8B5012202920022CDE90012694694
:10123000FFF7EAFB8FBDF8B5032203921122CDE937
:1012400000126946FFF7E0FB8FBD0000B0B5044611
:1012500000687C4D2169A28802614800A847FFF719
:1012600029FED4E90001FFF7E9FD04F1080207CAED
:101270000904016150002946BDE8B040084700BF9D
:10128000B0B5044600686F4D6168FFF7D7FDFFF702
:1012900011FE20682169A288026148002946BDE844
:1012A000B0400847B0B5044601680069A2880A61E9
:1012B000FFF76AFBFFF7B3FDD4E90001FFF7B1FFC9
:1012C000D4E9000100238AB28568154205D05D1C6F
:1012D000F92B2B4688BFB0BDF6E7FFF7ACFFD4E98A
:1012E0000212206912040A61BDE8B040FFF74CBB4E
:1012F000F8B505460C468068524F0026E968090497
:101300000161072E88BFF8BD60B2A988B0F1FF3F28
:10131000C8BF090428692A681161B8472869A96803
:10132000AA890A61B847D5E90212286912040A613C
:10133000B84701366400E4E710B586B0234C20447A
:101340004FEAB02003280FD8DFE800F002101E2C6F
:101350001F48046844F004040460006800F00400BE
:10136000FFF77DFD1B482AE000202CE018480468A8
:1013700044F008040460006800F00800FFF76FFD07
:10138000144800F580601AE01148046844F0100425
:101390000460006800F01000FFF761FD0D4800F5E3
:1013A00000600CE00A48046844F02004046000680F
:1013B00000F02000FFF753FD064800F5406002A949
:1013C000FFF722FB012006B010BD00BF00F8FEBFF2
:1013D00018100240000801402DE9F047DFF8649042
:1013E0008A4605464FF000080026072E26D8D5E984
:1013F0000012286A12040A61C8474FFA8AF0A989C4
:10140000B0F1FF3FC8BF0904286AAA681161C84744
:10141000286A2968AA880A61C847D5E90417286A92
:101420008C68C84707EA04004FEA4A0A80B20028DD
:1014300018BF012040EA48080136D6E75FFA88F075
:10144000BDE8F08789090008012181F31088002296
:101450002349096982F31088081A6FF00041B8BF68
:101460000844704720050020B0B51D48816801314F
:101470008160417891B3416929B141690139416184
:1014800004BF01218170714A0021012324290ED05B
:10149000541865684DB16568013D656005D163709C
:1014A000555C012D04BFA56865600C31EEE701694C
:1014B000013101610169013104BF00210161C1787D
:1014C0000131CAB2092A88BF0021C170C188013127
:1014D0008AB2D2087C2A88BF0021C180B0BD00BF7B
:1014E000200500200E480F4A016841F0010101600B
:1014F000416811400C4A4160016811400160016877
:1015000021F480210160416821F4FE0141604FF423
:101510001F01816005484FF000610160704700BF06
:10152000001002400000FFF8FFFFF6FE08ED00E0AB
:1015300070B5464C606A0668C5684169B10616D543
:101540004068E16A628F8854618F4A1C628792B258
:10155000618E8A4224BF00226287E28F8A4202D2D1
:10156000E18F0131E187216C09B1C0B288473006B3
:1015700018D5280616D5208F58B1012084F84400CC
:10158000FFF774FC24BF0020E086208F01382087FD
:1015900008E0606AC16821F08001C160C16841F063
:1015A0004001C16070060BD5680609D5208F40B197
:1015B000FFF75CFC24BF0020E086208F01382087E5
:1015C00070BD002084F84400606AC16821F04001C9
:1015D000C16070BDFEE7000078B51C4B0021012200
:1015E0000024012C2CD082F310881D8FADF80250FE
:1015F00081F310881D8EBDF80260AE420CD3BDF899
:101600000260AE42EFD15D6AEE683606EBD4EE685A
:1016100046F08006EE60E6E79D6A9E8EA85582F34E
:1016200010889D8E01359D86ADB21E8EB54228BFB5
:1016300099861D8F013401351D8781F31088D0E70D
:10164000596ACA6842F08002CA6078BD7C050020F1
:101650008AB07C4D7C4C4FF6FF01286840F01000AA
:101660002860206808407949084320600F20FFF770
:101670009FFA774E306800F00C00042819D03068CB
:1016800000F00C00082802D13068C00311D456F8CD
:10169000040C40F4803046F8040CDFF8AC06816896
:1016A00056F8042C920306D48268521A642AF7D999
:1016B0008EE056F8040C306800F00C00082862D167
:1016C000306800F47410B0F5E81F40F0818028689D
:1016D00010F0060F09D12868022161F3020028608A
:1016E000286800F00700022822D1306840F4E0604A
:1016F0003060306840F460503060306820F0F000B6
:10170000306056F8040C800112D530680221DFF8F1
:10171000387661F3010041F288313060B868326890
:1017200002F00C02082A06D0BA68121A8A42F6D9C8
:101730003320FFF745F9286800F00700032809D394
:101740002868022161F302002860286800F0070081
:101750000228EDD13068042161F30A20306030683E
:1017600020F4605030603B48316801F00C02082AD8
:101770003AD1C1F383420FF2D453C9039A5C2AD4FD
:101780003548504330E0354900200860DFF8B8059F
:10179000826856F8043C9B0104D583689B1A022B8F
:1017A000F7D915E0326822F400323260326822F450
:1017B000741202F5E812326001220A60816856F85C
:1017C000042C92013FF583AF8268521A022AF6D99F
:1017D0002720FFF7F5F8316850430FF28052C1F32C
:1017E0004041515CB0FBF1F031680FF27452DFF808
:1017F0008055C1F30311515CC8403978286010202E
:10180000002918BF0F20FFF7D3F970690222DFF813
:10181000647540F001007061706900F00100039090
:1018200003980F48016862F31A61016000200021EB
:10183000242917D07A1850609060507078540C3179
:10184000F6E700BF002002400CED00E00003FA05BF
:101850000410024000127A0000093D00600042427C
:101860000400014028684FF47A714FF0000BB0FB80
:10187000F1F003490138BBEB106F0AD102E000BF61
:1018800010E000E04860F020E0750720C1F808B0E3
:101890000860DFF8B4044FF00108DFF8DC14DFF86B
:1018A000DC24724D0DF10C0ADFF8D44480F801807D
:1018B0004FF00220A7F834B0A7F836B0A7F83AB036
:1018C000A7F83CB0A7F83EB0C7E9095287F844B082
:1018D000C7F840B0C7E90B10A7F838B05146706997
:1018E000FFF7D9FAFFF7D7FA40F4804070617069CA
:1018F00000F48040039003980320CDE90580022086
:1019000004904FF40070039059488146A0474FF46B
:101910008060514603904846A047252000210122BF
:10192000FFF76EF953484FF0200A41F20C610FF2B5
:1019300054423224C0F8F4A09DF8230024208DF8EE
:101940002300E86820F40050E860286920F4405043
:101950002861E86888430C30E860686920F44070CA
:101960006861DFF80C0400683168C1F3C221515C82
:10197000414AC840192148434FF4E121B0FBF1F13D
:10198000B0FBF2F06FF0630200FB0211642204EB83
:101990000111B1FBF2F101F0F00201F00F0102EBD5
:1019A0000010DFF8DC230844A860286920F4904088
:1019B0002861686920F02A006861E86840F40050F6
:1019C000E860CDF824B08DF823A08DF822A0286817
:1019D00020F040002860286820F020002860E86897
:1019E00040F02000E8604FF40055706940F01000AE
:1019F0007061706900F0100009900320CDE904883F
:101A000003950690099803A909F500609047DF48FF
:101A10003B46052240214560DD4D484688F310884D
:101A20007C60BC6087F801B087F800B080248BF33D
:101A3000108843F8489F4FF0100B4FF00809C3E996
:101A40000712C14AC3E903A0C3E90190C3E905B085
:101A5000824642F8404FC2E90410936150602A6008
:101A60000821FFF7E2F9C8B108E000BF00380140E3
:101A70000008014010E000E00020BF02D7E9140197
:101A8000FFF7D3F950B1D7E9160100220123FFF780
:101A900053FC18B1D7E91801FFF7C7F9706940F096
:101AA000040070617069564600F00400099003203C
:101AB00006900120CDE90340099803AC5046214629
:101AC000FEF7A2FF2868A04F4FF47F438169F960B9
:101AD0008A69898B1161AB82AF4BAE4A0021C5E99F
:101AE00002212B61018840680161FFF72DFA0AF598
:101AF00080663846052140F8186FC0E90196C0F8A5
:101B00000CB00161FFF748FB4FF4FA70FEF72AFFB3
:101B1000FEF7AAFEC0073FD107F118052846FFF7D8
:101B200095FBDFF8788228467021C0479C4F2846F5
:101B3000B8472846A821C0472846B847284600216C
:101B4000C0472846B84728460021C0472846B8471E
:101B50002846FFF795FB0A20FEF704FF2846FFF70B
:101B600075FB28467021C0472846B8472846BE2145
:101B7000C0472846B84728460821C0472846B847E6
:101B800028460021C0472846B8476F4F2846FFF730
:101B900077FB1420FEF7E6FE3D4605204FF400617A
:101BA0004FF4806245F82C6FC5E903102846C5E95B
:101BB0000126FFF7F1FA7B4E5020B0472846FFF789
:101BC00045FB28464621FFF793FB2846FFF76AFBB3
:101BD000284601214FF00108FFF78AFB2846FFF74E
:101BE00061FB2846FFF74CFB40208DF81C0032209B
:101BF0008DF80C00FEF74EFEFEF79CFE5020B0471D
:101C0000201D04F10801CDE90110FEF7A1FD6420BB
:101C1000B047FEF763FEDFF890A1644EDFF890B1A5
:101C20000DF124090690FEF735FEFEF783FE88F3DA
:101C3000108800203D6980F310882846FFF704FCD7
:101C40004F2837DC4846FFF705F80028F5D0014655
:101C5000032824D19DF824209DF825309DF82600E6
:101C6000232A08BF322B20D140281ED14749FFF735
:101C7000EAF858BF0420FFF705F94FF00008B8F163
:101C8000020FDAD8304600F091F92046FFF772F8DB
:101C90004FF49670FEF766FE08F10108EFE79DF835
:101CA00024209DF825309DF826000090584600F02D
:101CB00081F8C2E7DDE90110FEF74AFD4FF00108A7
:101CC00088F3108800203D6980F310882846FFF7CC
:101CD000BBFB632834DC4846FEF7BCFF0028F5D088
:101CE0000146032821D19DF824209DF825309DF838
:101CF0002600232A08BF322B1DD140281BD123499F
:101D0000FFF7A1F858BF0420FFF7BCF80027022F07
:101D1000DCD8304600F04AF92046FFF72BF84FF4A4
:101D20009670FEF71FFE0137F1E79DF824209DF81D
:101D300025309DF826000090584600F03BF8C5E796
:101D4000FEF7CCFD004F6DE72005002002030405DF
:101D5000060708090A0B0C0D0E0F101001020000F7
:101D6000000000000000000001020304060708094B
:101D7000040000207C05002008020020080000204C
:101D8000090A000800000000010203040C100140D1
:101D9000080400208050DE1901010700F11200083C
:101DA000A512000865090008F81F000817200008A0
:101DB000D91F00080FB4054B10B503A9044A0298B7
:101DC00000F018F810BC5DF814FB0000D9150008ED
:101DD0000000002002E008C8121F08C1002AFAD142
:101DE00070477047002001E001C1121F002AFBD19B
:101DF000704700002DE9FF4F8BB09A460F4605460D
:101E0000002606E025280BD052460D9990476D1C00
:101E1000761C28780028F5D10FB03046BDE8F08F49
:101E20000024A0460122604900E0044315F8013F68
:101E3000203B02FA03F00842F7D128782E2817D168
:101E400015F8010F44F004042A280ED06FF02F0279
:101E50002878A0F1300109290AD808EB880102EBA3
:101E6000410100EB01086D1CF2E757F8048B6D1C73
:101E7000287869283ED006DC0028CDD063280BD016
:101E8000642804D136E0732810D075284BD0524610
:101E90000D999047761C85E017F8040B8DF800002B
:101EA00000208DF80100E946012003E057F8049B6B
:101EB0004FF0FF3061074FF0000401D40AE0641CCA
:101EC00044450DDA8442FADB19F804100029F6D1F2
:101ED00006E0641C8442FCDB19F804100029F8D1E8
:101EE000264404E019F8010B52460D999047641EF0
:101EF000F8D257E001CF4FF00A0B002802DA404237
:101F00002D2102E0210504D52B218DF8241001217B
:101F100003E0E10705D02021F7E70DF12009089142
:101F20000CE00021F9E701CF4FF00A0BF9E7594621
:101F3000FEF7F8F801F1300209F8012D0028F6D17A
:101F4000ADEB090000F1200B600701D44FF0010850
:101F5000D84502DDA8EB0B0000E0002080460024FD
:101F600006E009A85246005D0D999047641C761C56
:101F700008988442F5DB04E0302052460D999047E2
:101F8000761CB8F10001A8F10108F5DC05E019F8AC
:101F9000010B52460D999047761CBBF10001ABF145
:101FA000010BF4DC6D1C34E70928010010B5044670
:101FB00001E0FFF711FB14F8010B04490028F8D1E8
:101FC000BDE810400A20FFF707BB0000000000201A
:101FD000060708090A0B0C01004765742057726F49
:101FE0006E6720436F6D6D616E645B25645D3A20A2
:101FF0002563256325630A00476574205269676875
:102000007420436F6D6D616E645B25645D3A2025BD
:1020100063256325630A0053656E64210000000098
:10202000402000080000002008000000D41D000827
:102030004820000808000020E01B0000E41D000804
:08204000000000000024F40080
:04000005080000ED02
:00000001FF
